:100000009E288030A100FE302D2001302D2075303B
:10001000A60030308528A101A117A900FE302D20AF
:1000200029082D28A400A700831605108312093083
:10003000A80003102220A70CA80B1A2803142220C2
:1000400024089928031827280000051029280514DA
:1000500029280030A6005B308528211B1228A70024
:10006000083024190130A800A70C220884002308B6
:10007000FF3A8005841780052308031880043C306C
:10008000842023088004A80B3428031499280830FE
:1000900024190130A800A701220884002308FF3A90
:1000A0008005841780052308800484130005FF3E23
:1000B000241DA70C2419A70D32308420A80B4E282C
:1000C000270803149928A400241C992822088400D6
:1000D0002308FF3A8005841780050130A600F4301C
:1000E0008520230880040130A600F4308528A8016B
:1000F000A700FF30A707031CA807031C992803309B
:10010000A600DF3085207928A601E83EA500A609D3
:10011000FC30031C8E28A50703188B28A5070000B8
:10012000A60F8B2825189428A51C9828000098282D
:10013000080083138312031300000800A00101309C
:10014000A8002C3078204030A10003204430122039
:10015000533012203230122034301220303012202E
:1001600035301220203012204E301220453012201F
:1001700054301220573012204F30122052301220AB
:100180004B301220203012205430122045301220E3
:1001900053301220543012200630A2008030A300C9
:1001A0000130A400632055302F2005302F20C530AA
:1001B0002F20C3302F2008302F2003012F200301D0
:1001C0002F2003012F20CD302F200630A2008030B9
:1001D000A3000430A4004720013903192A10031D8D
:1001E0002A142A1815294030A100C0300D205330A0
:1001F00012207730122069301220743012206330C0
:10020000122068301220203012202330122031308A
:100210001220203012203D301220203012204F308A
:10022000122046301220122037294030A100C03061
:100230000D20533012207730122069301220743094
:100240001220633012206830122020301220233018
:10025000122031301220203012203D301220203068
:1002600012204F3012204E30122020301220013048
:10027000A800F43078200630A2008030A3000130BE
:10028000A400632055302F2005302F20B3302F20BD
:10029000BF302F2008302F2003012F2003012F20F3
:1002A00003012F20AB302F200630A2008030A300A6
:1002B0000430A4004720013903192A10031D2A1411
:1002C0002A1884294030A10094300D205330122088
:1002D00077301220693012207430122063301220DF
:1002E00068301220203012202330122032301220A9
:1002F000203012203D301220203012204F301220AA
:10030000463012201220A6294030A10094300D2042
:1003100053301220773012206930122074301220AE
:100320006330122068301220203012202330122037
:1003300032301220203012203D3012202030122086
:100340004F3012204E301220203012200130A800F1
:10035000F43078200630A2008030A3000130A400E1
:10036000632055302F2005302F20B4302F20BF3090
:100370002F2008302F2003012F2003012F200301FD
:100380002F202E302F200630A2008030A300043012
:10039000A4004720013903192A10031D2A142A1822
:1003A000F3294030A100D4300D2053301220773093
:1003B000122069301220743012206330122068300D
:1003C000122020301220233012203330122020300F
:1003D00012203D301220203012204F3012204630A3
:1003E00012201220152A4030A100D4300D205330A5
:1003F00012207730122069301220743012206330BE
:100400001220683012202030122023301220333086
:100410001220203012203D301220203012204F3088
:1004200012204E301220203012200130A800F4306B
:080430007820CC2863001A2A91
:02400E00223F4F
:00000001FF
